:1010000039C000006DC000006BC0000069C0000066
:1010100067C0000065C0000063C0000061C0000040
:101020005FC000005DC000005BC00000F0C40000B5
:1010300057C0000055C0000053C0000051C0000060
:101040004FC000004DC00000F2C2000049C00000C7
:1010500047C0000045C0000043C0000041C0000080
:101060003FC000003DC000003BC0000039C0000090
:1010700037C0000011241FBECFEFD2E0DEBFCDBFCE
:101080002B9A8FE19EE40197F1F700C000001B9BB3
:1010900012C084B7877F84BF88E10FB6F89480932D
:1010A0006000109260000FBE1092A1011092A0018A
:1010B000E0E0F0E0099511E0A0E0B1E0EEE9FDE14B
:1010C00002C005900D92A239B107D9F711E0A2E94B
:1010D000B1E001C01D92A03AB107E1F731D05DC681
:1010E0008FCF84E08093E9008091E80085FD0EC0F9
:1010F0008091E8008B778093E8008091E80082FD82
:10110000F3CF8EB38111F9CF80E008958091F10083
:10111000089593E09093E9009091E80095FF03C053
:101120008093F10008959091E8009E779093E800F5
:101130009091E80090FDF4CF9EB39111F9CF0895FE
:10114000CF93DF9300D01F92CDB7DEB784B7877FF0
:1011500084BF88E10FB6F89480936000109260001D
:101160000FBE11E015BF82E085BF42D48AB1806F07
:101170008AB98BB18F708BB910936F0083E0809325
:1011800081008BB18F7080618BB97894A3E07A2E47
:10119000B5E06B2E212C312C80910001882309F4BD
:1011A0002FC284E08093E9008091E80082FF26C28C
:1011B00098DF982F853419F41092000107C088E851
:1011C000890F823010F0943521F48BDF8DE0A1DFA0
:1011D000EDC19035D9F39C34C9F3943721F484E4FC
:1011E00098DF80E0F4CF913611F489E5F0CF9134A7
:1011F00091F477DF082F75DF90E0880F991F202F7B
:1012000030E0322F2227330F822B932BAA2797FD12
:10121000A095BA2F9FC1903711F483E5D8CF9335AD
:1012200071F47AE8E72E71E0F72EF70181917F01E2
:1012300070DFF1E9EF16F1E0FF06B9F7B7C19635B7
:1012400021F481E366DF80E3C2CF933731F489E88C
:1012500060DF83E95EDF8EE1BACF9536A9F4E0E086
:10126000F0E070925700E89507B600FCFDCF609261
:101270005700E89507B600FCFDCFE058FF4FE11599
:1012800080E1F80771F7A2CF9C3651F42ADF8095F0
:1012900099E0E1E0F0E0082E90935700E89596CFB2
:1012A000923721F489E0E1E0F0E010C0963419F4BF
:1012B00089E0F1010BC09E3421F489E0E3E0F0E025
:1012C00005C0913539F489E0E2E0F0E08093570001
:1012D00084917DCF923631F489E51BDF80E019DF00
:1012E00080E875CF923419F0973609F0CEC0998313
:1012F000F8DEA82EB12CBA2CAA24F3DEA82AF1DE3F
:10130000082F8BEB800F9981823010F08FE35FCF35
:10131000973609F044C081E180935700E895450174
:10132000B12C8114910409F441C1C0909201D09074
:101330009301E0909401F09095010634B9F4EB2DFF
:10134000F0E0EC29FD298491E4DEBB2069F0F2E0B5
:10135000CF0ED11CE11CF11CC0929201D0929301DE
:10136000E0929401F0929501B12615C0D701C60113
:10137000B695A79597958795FAD4CBDE82E0C80EEF
:10138000D11CE11CF11CC0929201D0929301E09219
:101390009401F092950191E0891A9108C2CFC09012
:1013A0009201D0909301E0909401F0909501063461
:1013B00029F0BB82AA82412C512C31C0F6017092D7
:1013C0005700E89507B600FCFDCFF3CF063479F55A
:1013D000552051F18090920190909301A09094013A
:1013E000B09095017EDE242D30E0382BF401090108
:1013F00010935700E8951124F2E08F0E911CA11C68
:10140000B11C8092920190929301A0929401B092AB
:10141000950151268A819B8101979B838A83EA816A
:10142000FB81EF2B99F626C05CDE482EF2CF59DE09
:10143000682F8091920190919301A0919401B091B5
:101440009501B695A7959795879599D48091920126
:1014500090919301A0919401B09195010296A11DE4
:10146000B11D8093920190939301A0939401B09346
:101470009501D0CF063409F0A9CEF601609257004D
:10148000E89507B600FCFDCFA1CE933469F4E09057
:101490009201F090930125DE90E0F7010C0110938A
:1014A0005700E895112492CE9336F9F4C09092013A
:1014B000D0909301E0909401F090950112DEF60136
:1014C000E16090E00C0110935700E8951124F2E0E0
:1014D000CF0ED11CE11CF11CC0929201D09293015D
:1014E000E0929401F092950171CE9D3659F4E0910D
:1014F0009201F091930160925700E89507B600FCC5
:10150000FDCF64CE923551F4E0919201F0919301B8
:10151000E590F4908F2DFDDD8E2D59CE943419F584
:10152000E0DD682F8091920190919301A091940148
:10153000B0919501B695A7959795879520D4809100
:10154000920190919301A0919401B091950102961E
:10155000A11DB11D8093920190939301A0939401DA
:10156000B093950133CE9436F1F4C0909201D090AF
:101570009301E0909401F0909501D701C601B695D2
:10158000A79597958795F3D3C4DD82E0C80ED11C4B
:10159000E11CF11CC0929201D0929301E09294015F
:1015A000F092950103C09B3109F0B0CE7092E90032
:1015B0009091E8008091E8008E778093E80095FD97
:1015C00011C08091E80080FD04C08EB38111F9CF75
:1015D00015C08091E8008E778093E80003C08EB339
:1015E000882361F08091E80080FFF9CF94E0909328
:1015F000E9008091E8008B778093E8009DD3CCCD03
:101600008091E00081608093E00082E49CED909303
:10161000A1018093A0012CE088E190E00FB6F8943E
:10162000A895809360000FBE20936000FFCF1F92AB
:101630000F920FB60F9211248F9380E389B98F9187
:101640000F900FBE0F901F90189542E061EC82E062
:1016500069D142E161E883E065D142E160E884E07C
:1016600061C1809198018F778132D9F580E389B982
:1016700080919901813229F0823249F1803289F5D5
:1016800012C080919801813A61F58091E800877FCE
:101690008093E80067E070E081E091E0A8D080915D
:1016A000E8008B7711C0809198018132D1F480914C
:1016B000E800877F8093E80067E070E081E091E0D8
:1016C000F7D08091E8008E778093E80008958091AC
:1016D0009801813231F48091E800877F8093E8009F
:1016E00035C10895292F30E02230310539F02330FB
:1016F000310549F02130310561F410C08EE390E0EE
:101700002AE331E01EC0882371F0813089F08230F5
:10171000A1F080E090E020E030E013C082E190E0B2
:1017200028E731E00EC084E090E026E331E009C014
:1017300088E190E02CE131E004C082E190E028E013
:1017400031E0FA0131832083089507B600FCFDCF14
:10175000F999FECF23E0FB0120935700E89507B6E7
:1017600000FCFDCF81E180935700E895089507B60E
:1017700000FCFDCFF999FECF25E0FB012093570037
:10178000E89507B600FCFDCF81E180935700E8950E
:10179000089507B600FCFDCFF999FECF21E0FB01CB
:1017A0000A0120935700E8951124089521E2FC01D5
:1017B000209357008491089529E0FC01209357005D
:1017C00084910895E1E0F0E089E0809357008491EE
:1017D000089507B600FCFDCFF999FECF809599E0FA
:1017E000E1E0F0E0082E90935700E89508952091ED
:1017F0009E0130919F012617370748F0611571054A
:1018000039F42091E8002E772093E80001C0B90157
:1018100020E061157105C9F13EB3332309F442C0DC
:10182000353009F441C03091E80033FD3FC03091BC
:10183000E80032FF06C08091E80082FF29C080E006
:1018400008953091E80030FFE4CF2091F20030E0BD
:10185000FC01281B390BCF01820F931F6115710505
:1018600049F08830910530F481918093F100615006
:101870007109F1CF21E0089709F020E08091E8009C
:101880008E778093E800CF01C4CF2111C5CFD3CF8D
:101890008EB3882339F0853039F08091E80083FFDA
:1018A000CACF04C082E0089583E0089581E00895DE
:1018B0006115710529F42091E8002B772093E80049
:1018C0006115710511F12EB3222341F1253041F14B
:1018D0002091E80023FD1EC02091E80022FFF3CFF5
:1018E000FC01CF012091F200222329F38091F10025
:1018F0008193CF01615071096115710591F7DBCFBB
:101900008EB3882359F0853059F08091E80080FF2C
:10191000F7CF02C081E0089580E0089582E0089545
:1019200083E008958F708093E900EBEEF0E0808112
:1019300081608083EDEEF0E010826093EC004083E4
:101940008091EE00881F8827881F08958091980154
:1019500087FD05C08091E80080FF0DC010C0809118
:10196000E80082FD04C08EB38111F9CF0895809103
:10197000E8008B7707C08EB38111ECCF089580917A
:10198000E8008E778093E80008953BD03DD08091A9
:10199000D8008F778093D8008091D800806880939A
:1019A000D8008091D8008F7D8093D80019BC82E048
:1019B00089BD09B400FEFDCF1EBA1092960142E027
:1019C00060E080E0AFDF8091E1008E7F8093E100F6
:1019D0008091E20081608093E2008091E200886063
:1019E0008093E2008091E0008E7F8093E000089574
:1019F000E3E6F0E080818E7F808381E08093970131
:101A0000C4CF1092E20008951092E10008951F9251
:101A10000F920FB60F9211242F933F934F935F9322
:101A20006F937F938F939F93AF93BF93EF93FF93A6
:101A30008091E10080FF16C08091E20080FF12C01B
:101A40008091E2008E7F8093E2008091E2008061CD
:101A50008093E2008091D80080628093D80019BC06
:101A60001EBA69D18091E10084FF2DC08091E2000F
:101A700084FF29C019BC82E089BD09B400FEFDCFF6
:101A80008091D8008F7D8093D8008091E1008F7E77
:101A90008093E1008091E2008F7E8093E20080914C
:101AA000E20081608093E20080919601882311F02A
:101AB00084E007C08091E30087FF02C083E001C09B
:101AC00081E08EBB38D18091E10083FF21C08091FD
:101AD000E20083FF1DC08091E100877F8093E100D9
:101AE00082E08EBB109296018091E1008E7F809300
:101AF000E1008091E2008E7F8093E2008091E2001D
:101B000080618093E20042E060E080E00BDF13D16F
:101B1000FF91EF91BF91AF919F918F917F916F91C5
:101B20005F914F913F912F910F900FBE0F901F909B
:101B300018951F93CF93DF9300D0CDB7DEB7E8E9B8
:101B4000F1E08091F100819381E0E03AF807C9F774
:101B500088DD8091E80083FFDAC090919801809140
:101B60009901853009F465C030F4813059F168F08D
:101B7000833041F1CCC0883009F49CC0893009F42D
:101B8000ABC0863009F0C3C075C0903881F0923880
:101B900009F0BDC080919C018F708093E900909105
:101BA000EB0095FB992790F91092E90001C090E0B5
:101BB0008091E800877F8093E8009093F100109275
:101BC000F10083C0292F2D7F09F0A1C0923009F0C8
:101BD0009EC090919A01911126C020919C012F7076
:101BE00009F495C02093E9009091EB0090FF1BC091
:101BF000833021F48091EB00806213C08091EB0070
:101C000080618093EB0081E090E0022E01C0880F9C
:101C10000A94EAF78093EA001092EA008091EB00C0
:101C200088608093EB001092E9008091E800877F44
:101C30004FC091116CC010919A011F778091E30001
:101C40008078812B8093E3008091E800877F8093E8
:101C5000E8007CDE8091E80080FFFCCF8091E3000B
:101C600080688093E300112311F083E001C082E0DB
:101C70008EBB4DC09058923008F049C0AE014F5F06
:101C80005F4F60919C0180919A0190919B012ADDA8
:101C9000009709F43CC02091E800277F2093E800DA
:101CA000BC0189819A81A3DD8091E8008B778093C4
:101CB000E8002DC0903859F58091E800877F809327
:101CC000E800809196018093F1008091E8008E7782
:101CD0008093E8003BDE1BC0911119C090919A01DE
:101CE0009230A8F48091E800877F8093E800909379
:101CF00096012CDE80919601811104C08091E30051
:101D000087FF02C084E001C081E08EBB9EDC809131
:101D1000E80083FF0AC08091E800877F8093E80095
:101D20008091EB0080628093EB000F900F90DF9129
:101D3000CF911F9108950895CF938EB38823A9F072
:101D40008091E9008F709091EC0090FF02C090E8C4
:101D500001C090E0C92FC82B1092E9008091E800E3
:101D600083FDE7DECF70C093E900CF910895F99924
:101D7000FECF92BD81BDF89A992780B50895262F90
:101D8000F999FECF1FBA92BD81BD20BD0FB6F89460
:0E1D9000FA9AF99A0FBE01960895F894FFCFC3
:101D9E00010000000000000812034C005500460030
:101DAE00410020004300440043000000180344009B
:101DBE00650061006E002000430061006D0065004B
:101DCE007200610000000403090409023E000201D2
:101DDE0000803209040000010202010005240010F7
:101DEE0001042402020524060001070582030800EF
:101DFE00FF09040100020A0000000705040210009A
:101E0E0005070583021000051201100102000008EB
:101E1E00EB034A200001010200014C5546414344A8
:021E2E0043006F
:101FA000D4CBE5CBF6CB02CC07CC0CCC12CC08952D
:081FB0000895089508950895B5
:101FE000DFCFDFCFDFCFDFCFDFCFDFCFDFCFDFCF81
:081FF000DFCFDFCFDFCFDFCF31
:081FF8000010000000DFFBDC1B
:0400000300001000E9
:00000001FF
